:020000040800F2
:1000000070040020450100088D11000885110008CA
:1000100089110008350400089D1400080000000044
:10002000000000000000000000000000B9110008FE
:1000300039040008000000008F110008BB110008FF
:100040005F0100085F0100085F0100085F01000810
:100050005F0100085F0100085F0100085F01000800
:100060005F0100085F0100085F0100085F010008F0
:100070005F0100085F0100085F0100085F010008E0
:100080005F0100085F0100085F0100085F010008D0
:100090005F01000800000000000000005F01000890
:1000A0005F0100085F0100085F0100085F010008B0
:1000B0005F0100085F0100085F0100085F010008A0
:1000C0005F0100085F0100085F0100085F01000890
:1000D0005F0100085F0100085F0100085F01000880
:1000E0005F0100085F010008000000005F010008D8
:1000F0005F0100085F0100085F0100085F01000860
:100100005F0100085F0100085F0100085F0100084F
:100110005F0100085F0100085F0100085F0100083F
:100120005F0100085F0100085F0100085F0100082F
:10013000DFF80CD000F03CF800480047F914000844
:10014000700400200648804706480047FEE7FEE7A7
:10015000FEE7FEE7FEE7FEE7FEE7FEE7FEE7FEE777
:10016000C51100083101000840EA01039B0703D0D4
:1001700009E008C9121F08C0042AFAD203E011F8E6
:10018000013B00F8013B521EF9D27047D2B201E0A8
:1001900000F8012B491EFBD270470022F6E710B58C
:1001A00013460A4604461946FFF7F0FF204610BDE5
:1001B000064C074D06E0E06840F0010394E80700B4
:1001C00098471034AC42F6D3FFF7B6FF8416000808
:1001D000A416000800BFFEE710B500F0C9FA10BD74
:1001E00070B5C2B04822734930A8FFF7BDFF48215F
:1001F0001EA8FFF7D2FF28226E49483114A8FFF746
:10020000B3FF28226B4970310AA8FFF7ADFF282100
:100210006846FFF7C2FF00240026002566486749AC
:100220008860674888606748C8606748C8606748F2
:100230006749086067486149C1F88C0200BF16E051
:10024000032600BF30A850F824000568E84380B2B8
:10025000B0EB154F03D11EA840F8245002E0701EE9
:10026000061EEFD100BF0EB9FFF7B6FF641C122CBB
:10027000E6D31E98C0F30B001F99C1F30B0140EAAF
:10028000014000902098C0B20190219800F00F002A
:10029000229901F01F0140EA014002902398C0F327
:1002A0000A002499C1F30C0140EA0140039025980B
:1002B000C0F30A002699C1F30A0140EA0140049004
:1002C000279800F03F00289901F03F0140EA0140E3
:1002D0000590299800F03F000690DDE92A0161F3BE
:1002E0001F400790DDE92C0161F31F4008902E9814
:1002F000C0F30B002F99C1F30B0140EA01400990B4
:1003000000241BE014A850F8240005685DF82410B0
:100310000AA850F82400284081420ED014A850F8B2
:10032000240000680AA951F8241088435DF82410BD
:10033000084314A951F824100860641C0A2CE1D366
:1003400023488C38006840F001001C49C1F80002C5
:1003500000BF00BF00BF00BF00BF00BF00BF00BFA5
:1003600000BF00BF1548D0F8000220F0010013497B
:10037000C1F8000200240EE014A850F8240005681B
:100380005DF824100AA850F824002840814201D0CA
:10039000FFF722FF641C0A2CEED30848406940F0A6
:1003A0008040064948610846406940F00040486185
:1003B00042B070BDEC1500082301674500200240E3
:1003C000AB89EFCD3B2A19087F6E5D4C51407F5DB4
:1003D0008C2202406327CE4600B591B02C2106A89E
:1003E000FFF7DBFE142101A8FFF7D7FE1F200690C0
:1003F000002007900C9001200B90002009900D9098
:1004000001200E9006A800F001FB08B1FFF7E2FE04
:100410000F20019000200290039004904FF4806020
:100420000590002101A800F0B9F908B1FFF7D2FE4C
:1004300011B000BD00BFFEE77047000078B503466D
:100440000022CAE0012696400D6805EA0604002C49
:1004500071D04D68022D02D04D68122D13D1D608EF
:1004600003F1200555F826005507EE0E0F25B5407F
:10047000A8435607F60E0D69B5402843D60803F188
:10048000200545F82600186856000325B540A84306
:100490000D7905F003055600B540284318604D68F6
:1004A000012D08D04D68022D05D04D68112D02D0C8
:1004B0004D68122D13D1986856000325B540A84306
:1004C0005600CD68B540284398605868012595408E
:1004D000A8430D79C5F30015954028435860D868A6
:1004E00056000325B540A84356008D68B540284303
:1004F000D8604D6805F08055B5F1805F6CD100BFC4
:10050000394DAD6945F00105374EB5613546AD69E8
:1005100005F00105009500BF00BF344D960855F861
:10052000260095072E0F0F25B540A843B3F1904F35
:1005300002D1002515E04FE02D4DAB4201D1012540
:100540000FE02C4DAB4201D102250AE02A4DAB420F
:1005500001D1032505E0294DAB4201D1042500E07E
:1005600007259607360FB5402843204D960845F8D5
:100570002600234D2868A0434D6805F48035B5F565
:10058000803F00D120431E4D28602D1D2868A043C8
:100590004D6805F40035B5F5003F00D12043184DF6
:1005A0002D1D28602D1D2868A0434D6805F4801579
:1005B000B5F5801F00D12043114D083528602D1D51
:1005C0002868A0434D6805F40015B5F5001F00D15B
:1005D00020430B4D0C352860521C0D68D540002D72
:1005E0007FF430AF78BD00000010024014000140DD
:1005F0000004004800080048000C004800100048B3
:100600000004014001480068704700000400002019
:1006100003480068034909780844014908607047A5
:10062000040000200C00002010B5042000F08CF81D
:10063000072000F005F800F029F8002010BD0000A8
:1006400070B504460E4800784FF47A71B1FBF0F0B3
:100650000C490968B1FBF0F5284600F05BFC08B1D5
:10066000012070BD082C07D200222146501E00F048
:100670002DF80548046001E00120F2E70020F0E7D2
:100680000C000020000000200800002008B500BF7A
:100690000D48806940F001000B4988610846806977
:1006A00000F00100009000BF00BF00BF0846C06915
:1006B00040F08050C8610846C06900F0805000904A
:1006C00000BF00BF08BD0000001002402DE9F05F30
:1006D00080460D461646002700F0E2FE07463946E2
:1006E0002A46334601F00700C0F1070ABAF1030FAA
:1006F00002D94FF0030A01E0C0F1070AD14600F128
:10070000030ABAF1070F02D24FF0000A01E0A0F18C
:10071000040AD4464FF0010A0AFA09FAAAF1010ABA
:100720000AEA020A0AFA0CFA4FF0010B0BFA0CFB68
:10073000ABF1010B0BEA030B4AEA0B0421464046DE
:1007400000F0B6FEBDE8F09F00BF00F00702064BC8
:1007500019684FF6FF031940044B0B4343EA02218B
:10076000014B196000BF70470CED00E00000FA0576
:1007700000BFBFF34F8F0748006800F4E0600649F0
:100780000843001D03490860BFF34F8F00BF00BF3F
:1007900000BFFDE70CED00E00000FA0570B504466F
:1007A0000D460CB9012070BD5A48006800F00F00DA
:1007B000A8420ED25748006820F00F002843554940
:1007C00008600846006800F00F00A84201D0012030
:1007D000E9E7207800F0020002281DD1207800F01F
:1007E0000400042805D14C48406840F4E0604A49C0
:1007F0004860207800F00800082805D14648406885
:1008000040F46050444948604348406820F0F0009C
:10081000A168084340494860207800F0010078B39F
:100820006068012806D13C480068C0F3404090B998
:100830000120B8E76068022806D13748006800F058
:10084000807040B90120AEE733480068C0F3400033
:1008500008B90120A7E73048406820F0030061682C
:1008600008432D494860FFF7CDFE064609E0FFF733
:10087000C9FE801B41F28831884202D9032092E7E9
:1008800007E02548406800F00C006168B0EB810F7C
:10089000EDD12048006800F00F00A8420ED91D4895
:1008A000006820F00F0028431A49086008460068D5
:1008B00000F00F00A84201D0012074E7207800F07A
:1008C0000400042807D11448406820F4E060E1687F
:1008D000084311494860207800F00800082808D132
:1008E0000D48406820F46050216940EAC1000A497F
:1008F000486000F019F808494968C1F30311074A34
:10090000515CC8400649086006480068FFF798FE39
:10091000002048E70020024000100240D4150008E3
:1009200000000020080000202DE9F04192B0402294
:1009300022A102A8FFF718FC30A000680190002453
:10094000002500260027A0462D48446804F00C002E
:1009500060B3042802D0082827D102E0DFF8A48081
:1009600027E004F4701004F0C04140EAD11002A95D
:1009700001EB9040077804F44030B0F5803F04D09C
:1009800004F44030B0F5403F0AD11D484068C0F340
:10099000404001A90D5C1B487843B0FBF5F602E02E
:1009A000194807FB00F6B04603E000BFDFF85880A7
:1009B00000BF00BF404612B0BDE8F081020304054D
:1009C000060708090A0B0C0D0E0F1011121314154F
:1009D000161718191A1B1C1D1E1F2021222324253F
:1009E000262728292A2B2C2D2E2F3031323334352F
:1009F000363738393A3B3C3D3E3F3F3F010200002D
:100A00000010024000366E0100127A00F8B504466C
:100A10000CB90120F8BD207800F00100002873D047
:100A2000F748406800F00C00042813D0F4484068F0
:100A300000F00C00082818D1F148406800F480301C
:100A4000B0F5803F06D0EE48406800F48030B0F545
:100A5000403F0AD1EA480068C0F3404000286CD00B
:100A60006068002869D10120D4E76068B0F5803F54
:100A700007D1E348806B20F44070A1680843E04947
:100A8000886300BF6068B0F5803F06D1DC4800682D
:100A900040F48030DA49086028E0606858B9D848E6
:100AA000006820F48030D64908600846006820F4C9
:100AB000802008601AE06068B0F5A02F0BD1D04804
:100AC000006840F48020CE4908600846006840F481
:100AD000803008600AE0CA48006820F48030C849C5
:100AE00008600846006820F48020086000BF606845
:100AF00090B1FFF787FD054607E0FFF783FD401B38
:100B0000642802D9032085E717E0BD480068C0F3D8
:100B100040400028F1D010E0FFF774FD054606E0E4
:100B2000FFF770FD401B642801D9032072E7B44829
:100B30000068C0F340400028F2D1207800F00200A5
:100B4000022854D1AE48406800F00C0098B1AC487F
:100B5000406800F00C00082817D1A948406800F44C
:100B60008030B0F5803F10D0A548406800F4803058
:100B7000B0F5403F09D0A2480068C0F3400078B308
:100B80006069012833D0012044E76069B8B19C480E
:100B9000006840F001009A490860FFF733FD054600
:100BA00006E0FFF72FFD401B022801D9032031E7A3
:100BB00093480068C0F340000028F2D017E0904846
:100BC000006820F001008E490860FFF71BFD054614
:100BD00007E0FFF717FD401B022802D9032019E7A1
:100BE00005E087480068C0F340000028F1D1207874
:100BF00000F01000102830D1A069B8B18048806A98
:100C000040F010007E498862FFF7FCFC054606E0D4
:100C1000FFF7F8FC401B022801D90320FAE67848C8
:100C2000806AC0F340100028F2D016E07448806A51
:100C300020F0100072498862FFF7E4FC054606E0E8
:100C4000FFF7E0FC401B022801D90320E2E66C48D4
:100C5000806AC0F340100028F2D1207800F008002C
:100C6000082833D1E069D0B16548406A40F00100FE
:100C700063494862FFF7C6FC054606E0FFF7C2FC81
:100C8000401B022801D90320C4E65D48406AC0F336
:100C900040000028F2D0012000F07AFA16E058480F
:100CA000406A20F0010056494862FFF7ABFC054658
:100CB00006E0FFF7A7FC401B022801D90320A9E6A4
:100CC0004F48406AC0F340000028F2D1207800F07D
:100CD0000400042875D100274948C06900F08050FD
:100CE00070B900BF4648C06940F080504449C861AF
:100CF0000846C06900F08050009000BF00BF012787
:100D00004048006800F48070B0B93E48006840F484
:100D100080703C490860FFF775FC054606E0FFF768
:100D200071FC401B642801D9032073E63548006834
:100D300000F480700028F2D0E068012807D1304824
:100D4000006A20F01800216908432D49086200BF9D
:100D5000E068012806D12A48006A40F001002849CD
:100D6000086227E0E06858B92548006A20F00100D1
:100D7000234908620846006A20F00400086219E06E
:100D8000E06805280BD11E48006A40F004001C49A9
:100D900008620846006A40F0010008620AE018484C
:100DA000006A20F00100164908620846006A20F037
:100DB0000400086200BFE068A0B1FFF723FC05460D
:100DC00009E030E0FFF71EFC401B41F28831884209
:100DD00001D903201EE60A48006AC0F3400000283B
:100DE000F0D017E0FFF70EFC05460DE0FFF70AFC18
:100DF000401B41F28831884206D903200AE60000F0
:100E000000100240007000403F48006AC0F34000FC
:100E10000028EBD1012F05D13B48C06920F080505C
:100E20003949C86100BF206A90B33748406800F074
:100E30000C00082853D0206A022838D132480068B4
:100E400020F0807030490860FFF7DCFB054606E0C3
:100E5000FFF7D8FB401B022801D90320DAE52A4816
:100E60000068C0F340600028F2D1D4E909010843CA
:100E700025494968254A11400843234948600846E6
:100E8000006840F080700860FFF7BCFB054607E093
:100E900037E0FFF7B7FB401B022801D90320B9E573
:100EA00019480068C0F340600028F2D029E01648D5
:100EB000006820F0807014490860FFF7A3FB054626
:100EC00006E0FFF79FFB401B022801D90320A1E5A4
:100ED0000D480068C0F340600028F2D111E0206A9C
:100EE000012800D196E50848466806F48031606A1A
:100EF000814204D106483040A16A884201D00120D5
:100F000088E5002086E5000000100240FFFFC09F3A
:100F100000003C6070B504462546681EB0F1807F35
:100F200001D301200FE0681E4FF0E0214861072146
:100F30004FF0FF3000F0BCFA00204FF0E021886154
:100F400007200861002070BD70B504460D461646A6
:100F500000BF94F83C00012801D1022070BD01209F
:100F600084F83C0000BF022084F83D0036B1042E16
:100F70001BD0082E31D00C2E5ED145E029462068CA
:100F800000F0B0F92068806940F0080021688861AD
:100F90002068806920F004002168886120688069E9
:100FA000296908432168886147E02946206800F0E4
:100FB000D1F92068806940F4006021688861206868
:100FC000806920F4806021688861206880692969CF
:100FD00040EA0120216888612FE02946206800F05E
:100FE000F7F92068C06940F008002168C8612068EE
:100FF000C06920F004002168C8612068C0692969BF
:1010000008432168C86118E02946206800F01CFAEE
:101010002068C06940F400602168C8612068C06928
:1010200020F480602168C8612068C069296940EAAD
:1010300001202168C86100E000BF00BF012084F8E2
:101040003D0000BF002084F83C0000BF00BF85E7E2
:1010500010B504460CB9012010BD94F83D0028B924
:10106000002084F83C00204600F00CF8022084F8B0
:101070003D00211D206800F0B7F8012084F83D00F4
:101080000020E9E710B586B00446142101A8FFF757
:1010900084F800BF2448806940F4006022498861D8
:1010A0000846806900F40060009000BF00BF00BFE8
:1010B0000846406B40F0040048630846406B00F06F
:1010C0000400009000BF00BF0220029001200390A6
:1010D00002200490C00101900420059001A94FF066
:1010E0009040FFF7ABF94FF4007001900420059099
:1010F00001A94FF09040FFF7A1F94FF480600190F3
:101100000420059001A94FF09040FFF797F94FF4A4
:10111000006001900420059001A94FF09040FFF776
:101120008DF906B010BD00000010024070B50446F5
:101130000E4601223146206800F0C2F80F492068AF
:10114000884203D00E492068884201D1012000E086
:10115000002028B12068406C40F4004021684864B9
:101160002068806800F00705062D05D0206800681B
:1011700040F0010021680860002070BD002C014093
:101180000034014000BFFEE700BFFEE77047704734
:1011900008B508490968C9084FF47A72B1FBF2F141
:1011A0004143009100BF00BF00994A1E00920029F0
:1011B000F9D108BD00000020704710B5FFF728FAEC
:1011C00010BD000010B5FFF70BF80648006840F4AA
:1011D0007000044908604FF00060024980390860DF
:1011E00010BD000088ED00E010B50268294B984260
:1011F0000ED0B0F1804F0BD0274B984208D0274B30
:10120000984205D0264B984202D0264B984203D1F3
:1012100022F070024B681A431E4B984220D0B0F166
:10122000804F1DD01C4B98421AD01C4B984217D0AF
:101230001B4B984214D01B4B984211D01A4B98422A
:101240000ED01A4B98420BD0194B984208D0194B2C
:10125000984205D0184B984202D0184B984203D1BF
:1012600022F44072CB681A4322F080034C6943EAAF
:10127000040202608B68C3620B688362054B98426C
:1012800002D0084B984201D10B69036301234361EB
:1012900010BD0000002C0140000400400008004088
:1012A000000C004000340140004C0140005001405F
:1012B0000054014000180040001C00400020004085
:1012C00030B501F01F05012404FA05F3046A9C43BC
:1012D0000462046A01F01F0502FA05F52C4304625A
:1012E00030BD000030B5056A25F001050562026ACF
:1012F0004368846924F0700424F003040D682C43CF
:1013000022F002028D682A43104DA84200D103E06A
:101310000F4DA84206D100BF22F00802CD682A4333
:1013200022F00402094DA84202D0094DA84207D17B
:1013300023F4807323F400734D692B438D692B4391
:10134000436084614D684563026230BD002C0140FA
:101350000034014030B5056A25F010050562026AC7
:101360004368846924F4E04424F440740D6844EA3A
:10137000052422F020028D6842EA0512124DA8428F
:1013800000D103E0114DA84207D100BF22F0800236
:10139000CD6842EA051222F040020B4DA84202D06D
:1013A0000A4DA84209D123F4806323F400634D69F8
:1013B00043EA85038D6943EA8503436084614D6890
:1013C0008563026230BD0000002C01400034014002
:1013D00030B5056A25F480750562026A4368C46900
:1013E00024F0700424F003040D682C4322F40072EE
:1013F0008D6842EA0522124DA84200D103E0114D4A
:10140000A84207D100BF22F40062CD6842EA05225B
:1014100022F480620A4DA84202D00A4DA84209D1A6
:1014200023F4805323F400534D6943EA05138D6977
:1014300043EA05134360C4614D68C563026230BD71
:10144000002C01400034014030B5056A25F4805578
:101450000562036A4468C26922F4E04222F44072E1
:101460000D6842EA052223F400538D6843EA0533F0
:10147000084DA84202D0084DA84204D124F480446B
:101480004D6944EA85144460C2614D680564036295
:1014900030BD0000002C01400034014000BFFEE7D9
:1014A00002480068C0F30220704700000CED00E025
:1014B00010B5002804DB4A07130E054A135406E052
:1014C0004A07140E034A00F00F031B1FD45410BD2B
:1014D00000E400E018ED00E002E008C8121F08C1B7
:1014E000002AFAD170477047002001E001C1121FA5
:1014F000002AFBD170470000FFF796F8FEF76CFF5B
:1015000031483249086032213048C16040F21F3012
:101510002E49486000212D4801618160416181614F
:10152000FFF796FD08B1FEF755FE602028490860D8
:10153000002088600861C860886148610A204860AE
:1015400000222248FFF700FD08B1FEF743FE1420F9
:101550001F49486004221D48FFF7F6FC08B1FEF75A
:1015600039FE1E201A49486008221848FFF7ECFC93
:1015700008B1FEF72FFE2820154948600C221348B9
:10158000FFF7E2FC08B1FEF725FE00210F48FFF748
:10159000CDFD08B1FEF71EFE04210C48FFF7C6FD85
:1015A00008B1FEF717FE08210848FFF7BFFD08B194
:1015B000FEF710FE0C210548FFF7B8FD08B1FEF755
:1015C00009FE00BFFEE70000002C014010000020D3
:1015D0005000002000000000000000000102030491
:1015E0000607080900000000010203041051FF1F54
:1015F0001451FF1F1851FF1F4851FF1F4C51FF1F6F
:101600000056FF1F0456FF1F0052FF1F0452FF1F0A
:101610004051FF1F4451FF1F0852FF1F2051FF1F61
:101620002451FF1F2851FF1F2C51FF1F3051FF1F56
:101630003451FF1F082202400C22024020220240A7
:1016400028220240242202401C2202402C22024076
:10165000102202401422024018220240FF0FFF0F06
:10166000FF0000000F001F00FF07FF1FFF07FF071D
:101670003F003F003F000000FFFFFFFFFFFFFFFFB5
:10168000FF0FFF0FA416000800000020100000004C
:10169000D8140008B41600081000002060040000F0
:1016A000E814000800127A000000000008000000A2
:0416B0000100000035
:0400000508000131BD
:00000001FF
